:020000040000FA
:020000002528B1
:08000800A300030E8312A20005
:1000100005081839A0008B1C20288B102008031914
:100020002028183A03191C2810302005031D1A280F
:1000300002301E2801301E28033021068500A10051
:10004000220E8300A30E230E09008316FF239000C7
:100050009F01FC30850010308B00811395168312B0
:10006000073099000230A10085009F010508203962
:100070008316011703193D28011383128B178B1464
:1000800040284A344B342034543479347034653445
:10009000203446346C3469347034203446346C3443
:1000A0006F3470342E3420345034653474346534F5
:1000B00020344734723469346634663469347434B5
:1000C000683473342C3420344D3461347934203422
:1000D00032343034303434342E34203452343134E9
:0400E0002E34313455
:02400E00843FED
:00000001FF
